:1000000002006F3200000000000000020325000023
:10001000000000320000000000000032000000007C
:1000200000000032000000000000000000001EBEC2
:10003000FF011FEF4E22C395F022120036600350DD
:100040000122E422020047C3EDB50706ECB5060223
:10005000E42274012278EA7902D8FED9FC12002E3B
:1000600070F322E62401F6FA08E63400F64A227814
:100070007FE4F6D8FD75812F752000C28CE5895488
:10008000F02402F589758A06758C06D2B9D2AFD2F2
:10009000A975B070752200752300752500752600BE
:1000A000C206752400752A00C207752B00A296921D
:1000B0000450030200C5752C02752D0A75270875BA
:1000C000280C0200D1752C78752D3C7527087528F1
:1000D00008D28C7E2C7F01115575270F75280FA231
:1000E00091920440030200ED74010200EEE4C0E0CE
:1000F000A292920440030200FE74010200FFE4D0C9
:10010000F055F0B401028003020110711A02011CC3
:10011000A2929204500302011C752B05A2059204C1
:100120004003020309C205E524B400028003020172
:100130003775248002013A752400A291920450037D
:100140000201A4A29292045003020152752B0502EF
:1001500001A1E52BB4020280025003020167752B56
:1001600000752600752A00A29092045003020188AF
:10017000752B01852D2AE526B41E0280025003024C
:100180000185752B040201A1E52AB4000280030257
:10019000019B752B007526000201A1752B02782AA0
:1001A000160201B3E52BB40402800240030201B33E
:1001B000752B03C208E52BB4010280030201C4744D
:1001C000010201C5E4C0E0E52BB402028003020194
:1001D000D674010201D7E4D0F045F0B401028003E7
:1001E0000201F1E526B41902800250030201F1D2A6
:1001F00008E52BB40002800302020675270F75285C
:100200000FD294020294E52BB40102800302022F64
:1002100075F00AE52684C0F07827D0E0F675F00A7C
:10022000E52684C0E07828D0E0F6C294020294E586
:100230002BB402028003020252B207A207920450BA
:100240000302024702021075270F75280FC294029D
:100250000294E52BB40302800302026775270B7535
:10026000280AB294020294E52BB40402800302022D
:100270007C75270E75280E710C020294E52BB405CF
:1002800002800302029175270075280E710C02028C
:100290009402007B0525A208920440030202A47484
:1002A000010202A5E4C0E08525F0741E113A600346
:1002B0000202B874010202B9E4D0F055F0B40102B0
:1002C00080030202CAC2950202CCD295E525B52C64
:1002D000028003020309752500E52BB401028003A7
:1002E0000202E874010202E9E4C0E0E52BB4020274
:1002F00080030202FA74010202FBE4D0F045F0B47C
:1003000001028003020309052602011CA291920446
:100310005003020317711AB29422C2937E2C7F01FC
:100320001155D29322C0D0C2D3C0E0C0F0C083C068
:1003300082C000C001C002C003C004C005C006C026
:1003400007C008C009C00AC00BC00CC00DC00EC059
:100350000FC010C01175F070E52445F0C0E0782999
:10036000D0E0F68529B078221163AC22AD237ED08F
:100370007F0711446003020381752200752300D2B8
:1003800005A206920440030203A48528F0E5244553
:10039000F0C0E07829D0E0F675F050E52945F0F599
:1003A000B00203BB8527F0E52445F0C0E07829D0F2
:1003B000E0F675F060E52945F0F5B0B206D011D051
:1003C00010D00FD00ED00DD00CD00BD00AD009D049
:1003D00008D007D006D005D004D003D002D001D079
:1003E00000D082D083D0F0D0E0D0D0320000000026
:00000001FF
